 FETCE4B

 Timestamp is 407e00f2 (Thu Apr 15 11:26:42 2004)

 Preferred load address is 10000000

 Start         Length     Name                   Class
 0001:00000000 00000a64H .rdata                  CODE
 0001:00000a64 00000048H .rdata$debug            CODE
 0001:00000aac 00007cf2H .text                   CODE
 0001:000087a0 00000028H .idata$2                CODE
 0001:000087c8 00000014H .idata$3                CODE
 0001:000087dc 000000e4H .idata$4                CODE
 0001:000088c0 00000554H .idata$6                CODE
 0001:00008e20 0000004aH .edata                  CODE
 0002:00000000 000000e4H .idata$5                DATA
 0002:000000e8 00000154H .data                   DATA

  Address         Publics by Value              Rva+Base     Lib:Object

 0001:0000001c       ??_C@_1DO@CNOJ@?$AA?$FL?$AAV?$AAI?$AAA?$AAF?$AAE?$AAT?$AA?$FN?$AA?5?$AAv?$AAe?$AAr?$AAs?$AAi?$AAo?$AAn?$AA?5?$AA?3?$AA?5?$AA?$CF@ 1000101c     wince.obj
 0001:0000005c       ??_C@_19ELDJ@?$AA3?$AA?4?$AA3?$AA2?$AA?$AA@ 1000105c     wince.obj
 0001:00000068       ??_C@_1BI@OKED@?$AAA?$AAp?$AAr?$AA?5?$AA1?$AA5?$AA?5?$AA2?$AA0?$AA0?$AA4?$AA?$AA@ 10001068     wince.obj
 0001:00000080       ??_C@_1BC@HHPF@?$AA1?$AA1?$AA?3?$AA2?$AA5?$AA?3?$AA3?$AA3?$AA?$AA@ 10001080     wince.obj
 0001:00000494       ??_C@_1BK@MFHF@?$AAD?$AAe?$AAv?$AAi?$AAc?$AAe?$AAN?$AAu?$AAm?$AAb?$AAe?$AAr?$AA?$AA@ 10001494     registry.obj
 0001:000004b0       ??_C@_1BC@DMCG@?$AAD?$AAe?$AAv?$AAi?$AAc?$AAe?$AAI?$AAD?$AA?$AA@ 100014b0     registry.obj
 0001:000004c4       ??_C@_1BC@CENF@?$AAV?$AAe?$AAn?$AAd?$AAo?$AAr?$AAI?$AAD?$AA?$AA@ 100014c4     registry.obj
 0001:000004d8       ??_C@_1BG@FLPJ@?$AAV?$AAL?$AAA?$AAN?$AAI?$AAD?$AAL?$AAi?$AAs?$AAt?$AA?$AA@ 100014d8     registry.obj
 0001:000004f0       ??_C@_1BI@MBGK@?$AAN?$AAd?$AAi?$AAs?$AAV?$AAe?$AAr?$AAs?$AAi?$AAo?$AAn?$AA?$AA@ 100014f0     registry.obj
 0001:00000508       ??_C@_1BM@FJIP@?$AAP?$AAr?$AAo?$AAc?$AAe?$AAs?$AAs?$AAo?$AAr?$AAT?$AAy?$AAp?$AAe?$AA?$AA@ 10001508     registry.obj
 0001:00000524       ??_C@_1BI@FIFM@?$AAE?$AAn?$AAv?$AAi?$AAr?$AAo?$AAn?$AAm?$AAe?$AAn?$AAt?$AA?$AA@ 10001524     registry.obj
 0001:0000053c       ??_C@_1BC@FCLJ@?$AAC?$AAh?$AAe?$AAc?$AAk?$AAs?$AAu?$AAm?$AA?$AA@ 1000153c     registry.obj
 0001:00000550       ??_C@_1O@PECJ@?$AAV?$AAL?$AAA?$AAN?$AAI?$AAD?$AA?$AA@ 10001550     registry.obj
 0001:00000560       ??_C@_1BE@BDAO@?$AA8?$AA0?$AA2?$AA1?$AAp?$AAq?$AAt?$AAa?$AAg?$AA?$AA@ 10001560     registry.obj
 0001:00000574       ??_C@_1BG@JPJB@?$AAT?$AAx?$AAQ?$AAu?$AAe?$AAu?$AAe?$AAN?$AAu?$AAm?$AA?$AA@ 10001574     registry.obj
 0001:0000058c       ??_C@_1BI@ODIK@?$AAA?$AAd?$AAa?$AAp?$AAt?$AAi?$AAv?$AAe?$AAI?$AAn?$AAt?$AA?$AA@ 1000158c     registry.obj
 0001:000005a4       ??_C@_1CA@GCBL@?$AA2?$AAK?$AAS?$AAc?$AAa?$AAt?$AAt?$AAe?$AAr?$AAG?$AAa?$AAt?$AAh?$AAe?$AAr?$AA?$AA@ 100015a4     registry.obj
 0001:000005c4       ??_C@_17BHGN@?$AAP?$AAM?$AAC?$AA?$AA@ 100015c4     registry.obj
 0001:000005cc       ??_C@_1BC@PHKJ@?$AAF?$AAl?$AAo?$AAw?$AAC?$AAt?$AAr?$AAl?$AA?$AA@ 100015cc     registry.obj
 0001:000005e0       ??_C@_1BG@LFIM@?$AAH?$AAW?$AAP?$AAh?$AAy?$AAR?$AAe?$AAs?$AAe?$AAt?$AA?$AA@ 100015e0     registry.obj
 0001:000005f8       ??_C@_1BE@FONC@?$AAN?$AAw?$AAa?$AAy?$AAF?$AAo?$AAr?$AAc?$AAe?$AA?$AA@ 100015f8     registry.obj
 0001:0000060c       ??_C@_1BC@PDHL@?$AAW?$AAO?$AAL?$AAE?$AAv?$AAe?$AAn?$AAt?$AA?$AA@ 1000160c     registry.obj
 0001:00000620       ??_C@_1CE@OFKD@?$AAV?$AAa?$AAl?$AAi?$AAd?$AAa?$AAt?$AAe?$AAP?$AAa?$AAc?$AAk?$AAe?$AAt?$AAL?$AAe?$AAn?$AA?$AA@ 10001620     registry.obj
 0001:00000644       ??_C@_1BO@BJPG@?$AAC?$AAo?$AAn?$AAn?$AAe?$AAc?$AAt?$AAi?$AAo?$AAn?$AAT?$AAy?$AAp?$AAe?$AA?$AA@ 10001644     registry.obj
 0001:00000664       ??_C@_1BK@ECA@?$AAM?$AAa?$AAp?$AAR?$AAe?$AAg?$AAi?$AAs?$AAt?$AAe?$AAr?$AAs?$AA?$AA@ 10001664     registry.obj
 0001:00000680       ??_C@_1CE@PCMM@?$AAT?$AAr?$AAa?$AAn?$AAs?$AAm?$AAi?$AAt?$AAT?$AAh?$AAr?$AAe?$AAs?$AAh?$AAo?$AAl?$AAd?$AA?$AA@ 10001680     registry.obj
 0001:000006a4       ??_C@_1CC@BEPB@?$AAR?$AAe?$AAc?$AAe?$AAi?$AAv?$AAe?$AAT?$AAh?$AAr?$AAe?$AAs?$AAh?$AAo?$AAl?$AAd?$AA?$AA@ 100016a4     registry.obj
 0001:000006c8       ??_C@_1CA@PEBF@?$AAT?$AAr?$AAa?$AAn?$AAs?$AAm?$AAi?$AAt?$AAB?$AAu?$AAf?$AAf?$AAe?$AAr?$AAs?$AA?$AA@ 100016c8     registry.obj
 0001:000006e8       ??_C@_1BO@NHAK@?$AAR?$AAe?$AAc?$AAe?$AAi?$AAv?$AAe?$AAB?$AAu?$AAf?$AAf?$AAe?$AAr?$AAs?$AA?$AA@ 100016e8     registry.obj
 0001:00000708       ??_C@_1CK@NENP@?$AAR?$AAe?$AAc?$AAe?$AAi?$AAv?$AAe?$AAB?$AAu?$AAr?$AAs?$AAt?$AAI?$AAn?$AAd?$AAi?$AAc?$AAa?$AAt?$AAe@ 10001708     registry.obj
 0001:00000734       ??_C@_1BI@KNNM@?$AAB?$AAu?$AAr?$AAs?$AAt?$AAL?$AAe?$AAn?$AAg?$AAt?$AAh?$AA?$AA@ 10001734     registry.obj
 0001:0000074c       ??_C@_1BM@JACB@?$AAE?$AAa?$AAr?$AAl?$AAy?$AAT?$AAr?$AAa?$AAn?$AAs?$AAm?$AAi?$AAt?$AA?$AA@ 1000174c     registry.obj
 0001:00000768       ??_C@_1BK@IBCE@?$AAE?$AAa?$AAr?$AAl?$AAy?$AAR?$AAe?$AAc?$AAe?$AAi?$AAv?$AAe?$AA?$AA@ 10001768     registry.obj
 0001:00000784       ??_C@_1BO@DPB@?$AAF?$AAu?$AAn?$AAc?$AAt?$AAi?$AAo?$AAn?$AAN?$AAu?$AAm?$AAb?$AAe?$AAr?$AA?$AA@ 10001784     registry.obj
 0001:000007a4       ??_C@_1BG@LMJN@?$AAS?$AAl?$AAo?$AAt?$AAN?$AAu?$AAm?$AAb?$AAe?$AAr?$AA?$AA@ 100017a4     registry.obj
 0001:000007bc       ??_C@_1BE@GIME@?$AAB?$AAu?$AAs?$AAN?$AAu?$AAm?$AAb?$AAe?$AAr?$AA?$AA@ 100017bc     registry.obj
 0001:000007d0       ??_C@_1BI@KDJA@?$AAA?$AAd?$AAa?$AAp?$AAt?$AAe?$AAr?$AAT?$AAy?$AAp?$AAe?$AA?$AA@ 100017d0     registry.obj
 0001:000007e8       ??_C@_1BI@PJHC@?$AAA?$AAd?$AAa?$AAp?$AAt?$AAe?$AAr?$AAC?$AAF?$AAI?$AAD?$AA?$AA@ 100017e8     registry.obj
 0001:00000aac       _DllEntry                  10001aac f   wince.obj
 0001:00000ad3       _ETHbyGetHashIndexByCrc32  10001ad3 f   tether.obj
 0001:00000b01       _CRCdwCrc32                10001b01 f   tcrc.obj
 0001:00000b34       _CRCdwGetCrc32Ex           10001b34 f   tcrc.obj
 0001:00000b49       _MEMvAlign                 10001b49 f   tmem.obj
 0001:00000b97       _PCIXbFindDeviceInfo       10001b97 f   upcix.obj
 0001:00000d1b       _NPCIvRegBitsOn            10001d1b f   pcinet.obj
 0001:00000d5f       _NPCIvInitialize           10001d5f f   pcinet.obj
 0001:00000dc1       _MACbIsRegBitsOn           10001dc1 f   mac.obj
 0001:00000dda       _MACbIsRegBitsOff          10001dda f   mac.obj
 0001:00000def       _MACbyReadEECSR            10001def f   mac.obj
 0001:00000df7       _MACvWriteEECSR            10001df7 f   mac.obj
 0001:00000e31       _MACbyReadMIICR            10001e31 f   mac.obj
 0001:00000e39       _MACvReadISR               10001e39 f   mac.obj
 0001:00000e63       _MACvWriteISR              10001e63 f   mac.obj
 0001:00000e82       _MACvIntEnable             10001e82 f   mac.obj
 0001:00000e9f       _MACvIntDisable            10001e9f f   mac.obj
 0001:00000eb7       _MACbIsIntDisable          10001eb7 f   mac.obj
 0001:00000eda       _MACbyReadMultiAddr        10001eda f   mac.obj
 0001:00000ee9       _MACvWriteMultiAddr        10001ee9 f   mac.obj
 0001:00000efa       _MACvSetMultiAddrByHash    10001efa f   mac.obj
 0001:00000f35       _MACbyGetBootRomSize       10001f35 f   mac.obj
 0001:00000f40       _MACvGetForcedMediaType    10001f40 f   mac.obj
 0001:00000fd7       _MACvSetRxThreshold        10001fd7 f   mac.obj
 0001:00000ffe       _MACvSetTxThreshold        10001ffe f   mac.obj
 0001:00001025       _MACvGetTxThreshold        10002025 f   mac.obj
 0001:00001042       _MACvSetDmaLength          10002042 f   mac.obj
 0001:00001053       _MACvSetLoopbackMode       10002053 f   mac.obj
 0001:00001068       _MACvSetDuplexMode         10002068 f   mac.obj
 0001:000010a0       _MACbIsIn100MMode          100020a0 f   mac.obj
 0001:000010da       _MACvIsInFullDuplexMode    100020da f   mac.obj
 0001:000010f1       _MACbIsCableLinkOk         100020f1 f   mac.obj
 0001:00001102       _MACvSafeDisableMiiAutoPoll 10002102 f   mac.obj
 0001:00001147       _MACvEnableMiiAutoPoll     10002147 f   mac.obj
 0001:0000116d       _MACvSetPacketFilter       1000216d f   mac.obj
 0001:00001209       _MACvSaveContext           10002209 f   mac.obj
 0001:0000138c       _MACvRestoreContext        1000238c f   mac.obj
 0001:00001518       _MACvCompareContext        10002518 f   mac.obj
 0001:00001544       _MACvTimer0MiniSDelay      10002544 f   mac.obj
 0001:00001597       _MACvTimer0MicroSDelay     10002597 f   mac.obj
 0001:000015e5       _MACbSoftwareReset         100025e5 f   mac.obj
 0001:00001641       _MACbSafeSoftwareReset     10002641 f   mac.obj
 0001:00001684       _MACbSafeRxOff             10002684 f   mac.obj
 0001:000016ea       _MACbSafeTxOff             100026ea f   mac.obj
 0001:0000171b       _MACbStop                  1000271b f   mac.obj
 0001:0000173e       _MACbSafeStop              1000273e f   mac.obj
 0001:00001792       _MACbShutdown              10002792 f   mac.obj
 0001:000017d2       _MACvInitialize            100027d2 f   mac.obj
 0001:000018e6       _MACvReadHardwareMIBCounter 100028e6 f   mac.obj
 0001:0000190f       _MACvSetVCAM               1000290f f   mac.obj
 0001:0000195c       _MACvSetMCAM               1000295c f   mac.obj
 0001:000019b1       _MACvGetVCAM               100029b1 f   mac.obj
 0001:000019fe       _MACvGetMCAM               100029fe f   mac.obj
 0001:00001a53       _MACvSetMCAMMask           10002a53 f   mac.obj
 0001:00001a53       _MACvSetVCAMMask           10002a53 f   mac.obj
 0001:00001a69       _MACdwGetVCAMMask          10002a69 f   mac.obj
 0001:00001a7b       _MACdwGetMCAMMask          10002a7b f   mac.obj
 0001:00001a8d       _MACvSetTimer1ms           10002a8d f   mac.obj
 0001:00001ab2       _MACvSetTimer1us           10002ab2 f   mac.obj
 0001:00001ad7       _MIIbReadEmbeded           10002ad7 f   mii.obj
 0001:00001b3c       _MIIbWriteEmbeded          10002b3c f   mii.obj
 0001:00001b9f       _MIIbIsRegBitsOn           10002b9f f   mii.obj
 0001:00001bc9       _MIIbIsRegBitsOff          10002bc9 f   mii.obj
 0001:00001bef       _MIIvSetLoopbackMode       10002bef f   mii.obj
 0001:00001d10       _MIIbIsAutoNegotiationOn   10002d10 f   mii.obj
 0001:00001d28       _MIIbIsInFullDuplexMode    10002d28 f   mii.obj
 0001:00001e23       _MIIvInitialize            10002e23 f   mii.obj
 0001:00001f5b       _SROMvIssueDirect          10002f5b f   srom.obj
 0001:00001feb       _SROMwReadDirect           10002feb f   srom.obj
 0001:000020c1       _SROMbWriteDirect          100030c1 f   srom.obj
 0001:00002215       _CARDvSetMediaLinkMode     10003215 f   card.obj
 0001:0000245b       _CARDvSetLoopbackMode      1000345b f   card.obj
 0001:0000247f       _STAvClearAllCounter       1000347f f   mib.obj
 0001:0000248f       _STAvUpdateIsrStatCounter  1000348f f   mib.obj
 0001:000024b8       _STAvUpdateTallyCounter    100034b8 f   mib.obj
 0001:000024cd       _STAvUpdateRDStatCounter   100034cd f   mib.obj
 0001:0000264e       _STAvUpdateTDStatCounter   1000364e f   mib.obj
 0001:0000279d       _STAvUpdateHardwareMIBCounter 1000379d f   mib.obj
 0001:0000281d       _CPYvFromPacketToBuffer    1000381d f   copy.obj
 0001:00002981       _RGTvGetInfoFromRegistry   10003981 f   registry.obj
 0001:00002d1a       _MiniportShutdown          10003d1a f   isr.obj
 0001:00002d50       _MiniportEnableInterrupt   10003d50 f   isr.obj
 0001:00002e8c       _MiniportDisableInterrupt  10003e8c f   isr.obj
 0001:00002eab       _MiniportIsr               10003eab f   isr.obj
 0001:00002fdf       _MiniportHandleInterrupt   10003fdf f   dpc.obj
 0001:00003e8b       _MiniportSendPackets       10004e8b f   rxtx.obj
 0001:00003f25       _RXTXvSendQueuedPackets    10004f25 f   rxtx.obj
 0001:00003f97       _MiniportReturnPacket      10004f97 f   rxtx.obj
 0001:0000465b       _MiniportQueryInformation  1000565b f   info.obj
 0001:0000578d       _MiniportSetInformation    1000678d f   info.obj
 0001:000061d6       _BYTEvReverseForD          100071d6 f   info.obj
 0001:000061f1       _s_ChangeFilter            100071f1 f   info.obj
 0001:000062ee       _s_ChangeMulticastAddresses 100072ee f   info.obj
 0001:00006416       _ALCbAllocateRdTdMemory    10007416 f   alloc.obj
 0001:000064db       _ALCvFreeRdTdMemory        100074db f   alloc.obj
 0001:00006db1       _MINITimerSample           10007db1 f   timer.obj
 0001:00006fdc       _MiniportReset             10007fdc f   reset.obj
 0001:0000706c       _INIbInitAdapter           1000806c f   reset.obj
 0001:00007706       _INIvSetCorrectMediaMode   10008706 f   reset.obj
 0001:000078c9       _INIvCompleteAllBufPhysMap 100088c9 f   reset.obj
 0001:00007945       _INIvCompleteAllPendPkt    10008945 f   reset.obj
 0001:00007a06       _INIvCompleteAllQueuedPkt  10008a06 f   reset.obj
 0001:00007a6e       _INIvSafeResetRx           10008a6e f   reset.obj
 0001:00007ac8       _INIvSafeResetTx           10008ac8 f   reset.obj
 0001:00007bb2       _MiniportInitialize        10008bb2 f   init.obj
 0001:000085c1       _MiniportHalt              100095c1 f   init.obj
 0001:000086ce       _DriverEntry               100096ce f   main.obj
 0001:00008786       _NKDbgPrintfW              10009786 f   coredll:COREDLL.dll
 0001:0000878c       _NdisStallExecution        1000978c f   ndis:NDIS.dll
 0001:00008792       _NdisAdjustBufferLength    10009792 f   ndis:NDIS.dll
 0001:00008798       _NdisFlushBuffer           10009798 f   ndis:NDIS.dll
 0001:000087a0       __IMPORT_DESCRIPTOR_COREDLL 100097a0     coredll:COREDLL.dll
 0001:000087b4       __IMPORT_DESCRIPTOR_NDIS   100097b4     ndis:NDIS.dll
 0001:000087c8       __NULL_IMPORT_DESCRIPTOR   100097c8     coredll:COREDLL.dll
 0002:00000000       __imp__NKDbgPrintfW        1000a000     coredll:COREDLL.dll
 0002:00000004       \177COREDLL_NULL_THUNK_DATA 1000a004     coredll:COREDLL.dll
 0002:00000008       __imp__NdisWritePciSlotInformation 1000a008     ndis:NDIS.dll
 0002:0000000c       __imp__NdisStallExecution  1000a00c     ndis:NDIS.dll
 0002:00000010       __imp__NdisQueryBufferSafe 1000a010     ndis:NDIS.dll
 0002:00000014       __imp__NDIS_BUFFER_TO_SPAN_PAGES 1000a014     ndis:NDIS.dll
 0002:00000018       __imp__NdisReadPciSlotInformation 1000a018     ndis:NDIS.dll
 0002:0000001c       __imp__NdisQueryBufferOffset 1000a01c     ndis:NDIS.dll
 0002:00000020       __imp__NdisMCancelTimer    1000a020     ndis:NDIS.dll
 0002:00000024       __imp__NdisReleaseSpinLock 1000a024     ndis:NDIS.dll
 0002:00000028       __imp__NdisMSynchronizeWithInterrupt 1000a028     ndis:NDIS.dll
 0002:0000002c       __imp__NdisAcquireSpinLock 1000a02c     ndis:NDIS.dll
 0002:00000030       __imp__NdisUnchainBufferAtFront 1000a030     ndis:NDIS.dll
 0002:00000034       __imp__NdisAdjustBufferLength 1000a034     ndis:NDIS.dll
 0002:00000038       __imp__NdisFlushBuffer     1000a038     ndis:NDIS.dll
 0002:0000003c       __imp__NdisMCompleteBufferPhysicalMapping 1000a03c     ndis:NDIS.dll
 0002:00000040       __imp__NdisSetEvent        1000a040     ndis:NDIS.dll
 0002:00000044       __imp__NdisGetCurrentSystemTime 1000a044     ndis:NDIS.dll
 0002:00000048       __imp__NdisMStartBufferPhysicalMapping 1000a048     ndis:NDIS.dll
 0002:0000004c       __imp__NdisAllocateMemoryWithTag 1000a04c     ndis:NDIS.dll
 0002:00000050       __imp__NdisAllocateBufferPool 1000a050     ndis:NDIS.dll
 0002:00000054       __imp__NdisAllocatePacketPool 1000a054     ndis:NDIS.dll
 0002:00000058       __imp__NdisFreeMemory      1000a058     ndis:NDIS.dll
 0002:0000005c       __imp__NdisFreeBufferPool  1000a05c     ndis:NDIS.dll
 0002:00000060       __imp__NdisFreePacketPool  1000a060     ndis:NDIS.dll
 0002:00000064       __imp__NdisAllocatePacket  1000a064     ndis:NDIS.dll
 0002:00000068       __imp__NdisAllocateBuffer  1000a068     ndis:NDIS.dll
 0002:0000006c       __imp__NdisFreePacket      1000a06c     ndis:NDIS.dll
 0002:00000070       __imp__NdisFreeBuffer      1000a070     ndis:NDIS.dll
 0002:00000074       __imp__NdisMAllocateSharedMemory 1000a074     ndis:NDIS.dll
 0002:00000078       __imp__NdisMFreeSharedMemory 1000a078     ndis:NDIS.dll
 0002:0000007c       __imp__NdisSetTimer        1000a07c     ndis:NDIS.dll
 0002:00000080       __imp__NdisInitializeEvent 1000a080     ndis:NDIS.dll
 0002:00000084       __imp__NdisMInitializeTimer 1000a084     ndis:NDIS.dll
 0002:00000088       __imp__NdisMRegisterAdapterShutdownHandler 1000a088     ndis:NDIS.dll
 0002:0000008c       __imp__NdisMRegisterInterrupt 1000a08c     ndis:NDIS.dll
 0002:00000090       __imp__NdisAllocateSpinLock 1000a090     ndis:NDIS.dll
 0002:00000094       __imp__NdisMAllocateMapRegisters 1000a094     ndis:NDIS.dll
 0002:00000098       __imp__NdisMDeregisterIoPortRange 1000a098     ndis:NDIS.dll
 0002:0000009c       __imp__NdisMMapIoSpace     1000a09c     ndis:NDIS.dll
 0002:000000a0       __imp__NdisMRegisterIoPortRange 1000a0a0     ndis:NDIS.dll
 0002:000000a4       __imp__NdisMSetAttributesEx 1000a0a4     ndis:NDIS.dll
 0002:000000a8       __imp__NdisReadNetworkAddress 1000a0a8     ndis:NDIS.dll
 0002:000000ac       __imp__NdisCloseConfiguration 1000a0ac     ndis:NDIS.dll
 0002:000000b0       __imp__NdisReadConfiguration 1000a0b0     ndis:NDIS.dll
 0002:000000b4       __imp__NdisOpenConfiguration 1000a0b4     ndis:NDIS.dll
 0002:000000b8       __imp__NdisMQueryAdapterResources 1000a0b8     ndis:NDIS.dll
 0002:000000bc       __imp__NdisMUnmapIoSpace   1000a0bc     ndis:NDIS.dll
 0002:000000c0       __imp__NdisMFreeMapRegisters 1000a0c0     ndis:NDIS.dll
 0002:000000c4       __imp__NdisFreeSpinLock    1000a0c4     ndis:NDIS.dll
 0002:000000c8       __imp__NdisMDeregisterInterrupt 1000a0c8     ndis:NDIS.dll
 0002:000000cc       __imp__NdisMDeregisterAdapterShutdownHandler 1000a0cc     ndis:NDIS.dll
 0002:000000d0       __imp__NdisWaitEvent       1000a0d0     ndis:NDIS.dll
 0002:000000d4       __imp__NdisTerminateWrapper 1000a0d4     ndis:NDIS.dll
 0002:000000d8       __imp__NdisMRegisterMiniport 1000a0d8     ndis:NDIS.dll
 0002:000000dc       __imp__NdisInitializeWrapper 1000a0dc     ndis:NDIS.dll
 0002:000000e0       \177NDIS_NULL_THUNK_DATA   1000a0e0     ndis:NDIS.dll
 0002:000000e8       _RegistryString            1000a0e8     registry.obj
 0002:000001c0       _GlobalString              1000a1c0     registry.obj
 0002:000001d8       _VLANIDListString          1000a1d8     registry.obj
 0002:000001e0       _CERegString               1000a1e0     registry.obj

 entry point at        0001:00000aac

 Static symbols

 0001:000031a9       _s_vSyncClearIsr           100041a9 f   dpc.obj
 0001:000031e4       _ISRvProcessReceiveDescRing 100041e4 f   dpc.obj
 0001:00003ae4       _ISRvProcessTransmitDescRing 10004ae4 f   dpc.obj
 0001:00004059       _s_nsSendPacket            10005059 f   rxtx.obj
 0001:00006128       _s_dwGenPatCrc             10007128 f   info.obj
 0001:00006578       _ALCbAllocRdMemory         10007578 f   alloc.obj
 0001:00006982       _ALCvFreeRdMemory          10007982 f   alloc.obj
 0001:00006ac3       _ALCbAllocTdMemory         10007ac3 f   alloc.obj
 0001:00006ca1       _ALCvFreeTdMemory          10007ca1 f   alloc.obj
 0001:00006d38       _ALCbAllocateSharedMemory  10007d38 f   alloc.obj
 0001:00006d90       _ALCvFreeSharedMemory      10007d90 f   alloc.obj
 0001:00007b6b       _s_byCalcFlowResolution    10008b6b f   reset.obj
 0001:00008490       _s_FindPciConfiguration    10009490 f   init.obj
 0001:0000852b       _s_vFreeAdapterResources   1000952b f   init.obj
